:1000000080316E28080008007E14803100308600A0
:10001000003087000B1F0D280E2853282100931D48
:100020001228132853282000931D17281828532816
:100030008B31FA2380310130F5070A307502031C39
:1000400022282328272801302000BA00F5012000AB
:100050000C192B282C282F280130F30045280E18C6
:100060003228332836280230F30045288D1A3928E3
:100070003A283D280330F30045280D1B402841282D
:1000800044280430F3004528F3017408031D49286F
:100090004A285128730803194E284F2851287308FD
:1000A000B9007308F4008B1D562857286C280B1CC8
:1000B0005A285B286C288B31A12380310130210024
:1000C0009D008130220097008C3020009E00270088
:1000D00095018631162680317E1009008031702806
:1000E0008731FF278031EB0002308400213085000A
:1000F000EE30FE000230FF008B31C7238031F0016B
:10010000F101F201F301F401F50120308400003027
:1001100085002530FE000030FF008B31C723803181
:100120007E102000803194282000E0018D31682568
:1001300080312000B0018531C92580318C3020000C
:100140009E0003309F008431B72480318B170B173A
:1001500020003A080319AD28AE280029BA01013061
:10016000B8070A303802031CB628B728F028B801AF
:100170003008031DBC28BD28DB280130AA07003049
:10018000AB3D370A0319C528C628C8280130B70770
:100190002B08D8002A08D7008331D32380310A30B6
:1001A00020003702031CD528D628E82837088D31CF
:1001B000BC258031E82802303006031DE028E12804
:1001C000E8282D08D8002C08D7008D31D92580319A
:1001D000200034080319ED28EE28F0280130B4027D
:1001E0003008031DF428F52800298F316B27803152
:1001F00020004608A7004508A60084315424803119
:1002000020003908031905290629172A3C30B400B3
:10021000DD29300803190D290E2911298D311E25DC
:1002200080318431B7248031EB298B31AA2380318E
:10023000EB290230B0008C3190248031EB298C31D5
:10024000A3248031EB298B3183238031EB298B313F
:100250008A238031EB298D31842580318D311E2513
:100260008031EB293008003A03191529013A0319A6
:100270001929033A03191F29013A03192329073AB7
:1002800003192729013A03192B29033A03191529C0
:1002900015293508F63E860087012230873D010882
:1002A000031953295429EB293608031D58295929C4
:1002B0005C29FA30B6006729FA303602031C61293E
:1002C000622965293508B60067290130B6028631F2
:1002D00060268031EB2982316B228031EB296B085B
:1002E00003197329742976290130EB028F313F27D6
:1002F0008031EB2900302102C83003192002031C91
:100300008229832987296430A0020030A13B8D31E6
:100310004F258031EB298C31F324803111293008AD
:10032000013A03194929023A03196B29073A0319BB
:100330006F29013A03197A29033A03198B29EB290A
:100340000130B607FB303602031CA729A829A929CA
:10035000B6013608F63E860087012230873D010847
:10036000031DB329B4296729592902306B020318E8
:10037000BA29BB2976290130EB077629633021029F
:100380003930031920020318C629C7298729643088
:10039000A0070030A13D87293008013A0319A029A0
:1003A000023A03196B29073A0319B529013A0319CF
:1003B000BE29033A03198B29EB293908013A03199D
:1003C000CC29033A03198F29013A03193229073A34
:1003D00003190929EB29C8302000B100B9012B2AE3
:1003E00087319B27803120005708AD005608AC00AC
:1003F000232A2D08CC002C08CB00833152238031D6
:10040000232A34080319052A062A102A2D08CD00AC
:100410002C08CC000830CE008631E7268031232A14
:100420000030C500C6008D31A0258031232A600828
:10043000E00A003A0319F029013A0319F929033AAD
:100440000319012A232A033020006002031C292AF1
:100450002A2A2B2AE001340803192F2A302AA82837
:100460006B03031D342A352A4B2A442A0130B1027A
:1004700022000E15A630890B3B2A003222000E11F5
:10048000A630890B412A003220003108031D492A79
:100490004A2A362AA82802306B06031D502A512A00
:1004A000A828622A0130B10222008E100E15A63053
:1004B000890B582A003222008E140E11A630890BA7
:1004C0005F2A003220003108031D672A682A522A59
:1004D000A82880316E282000DD018C31352482313E
:1004E000003A0319742A752A6D2A64302000C50069
:1004F0000030C6002108C8002008C7008731262721
:100500008231200045088B31BD2382312000DE017D
:100510005E08F63E860087012230873D01080319F8
:10052000922A932AFF2A0130DD078C31352482314B
:10053000003A03199C2A9D2A952A20005E08D700BC
:10054000D801D735D80D0230D9002130DA0057084C
:100550005907860058085A3D8700403FDB00413F5D
:10056000DC005C088B31BD23823103302000D700D2
:100570009730890BB92AD70BB92A00328C31352430
:100580008231003A0319C52AC62ABE2A20005E0815
:10059000D700D801D735D80D0230D9002130DA0084
:1005A00057085907860058085A3D870001088B31C3
:1005B000BD23823103302000D7009730890BDE2A1B
:1005C000D70BDE2A00328C3135248231003A0319F0
:1005D000EA2AEB2AE32A20005E08F63E860087011D
:1005E0002230873D01088B31BD238231013020004C
:1005F000DE07FA305E02031CFE2AFF2A882A5930E1
:10060000CE009030CF008C31262482313C30200047
:10061000CC005D08D700D8015708CD005808CE009F
:1006200085317325823140302000C8008D31F82596
:1006300082318C3135248231003A0319202B212B51
:10064000192B20002B088B31BD2382310330200071
:10065000D7009730890B2A2BD70B2A2B00328C31ED
:1006600035248231003A0319362B372B2F2B2000EB
:100670002A088B31BD23823103302000D700973008
:10068000890B402BD70B402B00328C313524823123
:10069000003A03194C2B4D2B452B00308B31BD23D9
:1006A00082310800133020004C02893003194B02BC
:1006B000031C5B2B5C2B602B8830CB001330CC00F1
:1006C00011304C02313003194B020318682B692B8F
:1006D000802B0130CF008C30D100B930D2004C08D3
:1006E000C6004B08C5000A30C7000030C8008E3174
:1006F0001826833120004508D1024608D23B952BAD
:10070000CF01FE30D100F130D2004C08C6004B08BA
:10071000C5000C30C7000030C8008E311826833168
:1007200020004508D1024608D23B0930D236D10C10
:10073000890B962B00305202403003195102031CE2
:10074000A22BA32BA72B3F30D1000030D200383092
:100750008F311527833139308F31152783312000B0
:1007600051080F39D0007030D00750088F3115274D
:10077000833120005208CE005108CD000430CE361F
:10078000CD0C890BBF2B4D08D0004F080319C92B86
:10079000CA2BCC2B0430D0075030D00750088F31F3
:1007A00015278331080010302000C5000E30C60028
:1007B0005808C8005708C700873126278331200012
:1007C0004608DA004508D9003C30CC005A08CE0073
:1007D0005908CD0085317325833142302000CE0089
:1007E0008B31D323833167302000C8009030C9009B
:1007F0008D313625833120005A08C6005908C500BE
:100800001030C7000E30C8008E311826833120000A
:100810004508D7024608D83B3C30C5000030C6002A
:100820005808C8005708C7008731262783312000A1
:100830004608DA004508D9003C30CC005A08CE0002
:100840005908CD0085317325833142302000C8001E
:100850008D31F825833167302000C8009030C90001
:100860008D31362583313C302000C5000030C60074
:100870005808C8005708C7008F31992783312000D6
:100880004608DA004508D9003C30CC005A08CE00B2
:100890005908CD0085317325833142302000C800CE
:1008A0008D31F82583310800200033080319592CB5
:1008B0005A2C8B2C20087002D7002108713BD800DD
:1008C00058082702031D662C570826020318692CB6
:1008D0006A2C7C2CB3017108A5007008A4003C3080
:1008E000CC002508CE002408CD0085317325843145
:1008F0008631A5268431B62C27087102031D822C6F
:10090000260870020318852C862CB62C2708F100C7
:100910002608F000B62C20087007D7002108713D8A
:10092000D80027085802031D972C260857020318E1
:100930009A2C9B2CAB2C0130B3007108A3007008DB
:10094000A2003C30CC002308CE002208CD00853127
:1009500073258431782C71082702031DB12C70088F
:1009600026020318B42CB52CB62C862C08002700C0
:10097000950122008C122000B001AA01AB01B80140
:10098000B701A601A701F001F101A401A501A2018F
:10099000A3010130B300F201A801A901B101B60120
:1009A000FA303602031CD52CD62CD72CED2C360869
:1009B000F63E860087012230873D81013635023EB2
:1009C000860087012130873D36350030873D003075
:1009D000C03FC13F0130B607D02CB601B5013C3055
:1009E000B40000308B31ED238431A53A031DF92C7E
:1009F000FA2C042D01308E3159268431200047080D
:100A0000A1004608A000192DA5302000C500003027
:100A10008E317C268431F4302000C8000130C900BA
:100A200001308C31DE248431F4302000A00001300C
:100A3000A100080000302000D4000030D3000030B6
:100A4000D2000030D1004C084B044A044904031979
:100A50002A2D2B2D6A2D0130D500372D0130C935B7
:100A6000CA0DCB0DCC0D890B2F2D0130D507CC1F16
:100A70003A2D3B2D2E2D0130D135D20DD30DD40D75
:100A8000890B3C2D4C085002031D502D4B084F0282
:100A9000031D502D4A084E02031D502D49084D02DA
:100AA000031C532D542D5D2D4908CD024A08CE3B21
:100AB0004B08CF3B4C08D03B51140130CC36CB0C0B
:100AC000CA0CC90C890B5E2D0130D502031D692D9E
:100AD0006A2D3B2D5408CC005308CB005208CA00A5
:100AE0005108C900080007302000D6000A30C500B0
:100AF0000030C6004E08C8004D08C7008F31992746
:100B0000853120004508D5000A30C5000030C600F8
:100B10004E08C8004D08C7008731262785312000C0
:100B20004608CE004508CD00073056060319992D1A
:100B30009B2D01309C2D0030CF00D0014F08550473
:100B4000D1005008D2004D085104D3004E08520481
:100B5000D400530854040319AE2DAF2DB72D4C0803
:100B60005607860087015508303E8100BD2D4C0890
:100B700056078600870120308100FF30D607D61F38
:100B8000C22DC32D762D4C08083E860087018101B9
:100B900008008B315223853122000E128E11D03085
:100BA0002000C900C930890BD32DC90BD32D0032C9
:100BB0000C308F311527853138308F31152785312D
:100BC00039308F311527853114308F311527853114
:100BD00076308F311527853155308F311527853186
:100BE0006C308F311527853168302000C900E43022
:100BF000890BF82DC90BF82D000038308F311527DF
:100C000085310C308F311527853101308F31152713
:100C1000853103302000CA000830C9007730890BC5
:100C20000F2EC90B0F2ECA0B0F2E08008B314E232F
:100C3000863122000E128E11D030FA00CA30890B94
:100C40001F2EFA0B1F2E0C308E31A0268631383025
:100C50008E31A026863139308E31A026863114306F
:100C60008E31A026863176308E31A02686315530E1
:100C70008E31A02686316C308E31A02686316830C8
:100C8000FA00E430890B422EFA0B422E0032383043
:100C90008E31A02686310C308E31A026863101306F
:100CA0008E31A02686310330FB000830FA00773001
:100CB000890B582EFA0B582EFB0B582E00000800FB
:100CC000FA3020003606031D662E672E832E633011
:100CD000CE009030CF008C31172486313C3020007C
:100CE000CC002908CE002808CD0085317325863137
:100CF0003F302000C8008D31F825863172088D31D3
:100D0000BC258631A42E3608DB00DC01DB35DC0D8A
:100D10000230DD002130DE005B085D0786005C08E4
:100D20005E3D8700403FD700413FD8008331D32349
:100D3000863120003608F63E860087012230873D46
:100D400001088D31BC25863108000A3020003702A9
:100D5000031CAB2EAC2ED92E3635023E8600870101
:100D60002130873D36350030873D2A08C03F2B08AB
:100D7000C13F3608F63E860087012230873D37089E
:100D800081003608B500370872020318C82EC92E34
:100D9000CB2E3708F2000130A8070030A93D013002
:100DA000B607FA303606031DD62ED72ED92E0130BF
:100DB000B6023C30CE008B31E0238631200027087C
:100DC000F1002608F000B701C830B10008000A3071
:100DD00020004D02293003194C020318F02EF12E89
:100DE000F62E6430CF000030D000112FF030CF004D
:100DF0000A30D0004C08D83EC500F5304D3DC60045
:100E00005008C8004F08C7008731262786312000C8
:100E10004608D0004508CF000330CF35D00D890BF0
:100E20000D2F00305002653003194F02031C192F9B
:100E30001A2F1E2F6430CF000030D0005008C6009B
:100E40004F08C5008D31A025863108002000C9015A
:100E5000CA014508460403192E2F2F2F5C2F01309D
:100E6000CB00392F0130C535C60D890B332F01302A
:100E7000CB07C61F3C2F3D2F322F0130C935CA0D7D
:100E8000890B3E2F46084802031D482F450847029C
:100E9000031C4B2F4C2F512F4508C7024608C83B57
:100EA00049140130C636C50C890B522F0130CB02D4
:100EB000031D5B2F5C2F3D2F4A08C6004908C50063
:100EC00008002000C5008030C600822F21000E12CD
:100ED00020004608450503196E2F6F2F722F210041
:100EE0008E15742F21008E11003200320310200065
:100EF000C60C21000E1620000E1E7F2F802F7B2F88
:100F00000032003220004608031D872F882F662FED
:100F100021000E128E150032003221000E16200024
:100F20000E1E932F942F8F2F0032003221000E12AD
:100F300000320032080000302000DF000F30DE00F9
:100F4000FC30DD000030DC001F308E313826873168
:100F500020004508D8004608D900DA01DB015B080B
:100F6000CC005A08CB005908CA005808C9005F08CD
:100F7000D0005E08CF005D08CE005C08CD00853152
:100F80001A25873120004C08DF004B08DE004A0894
:100F9000DD004908DC005D08D7005C08D6000800C9
:100FA00022008C018D0118308E001F3021008C0032
:100FB000F0308D0039308E00C63023008E001030A6
:100FC0008D0003308C00603024008D0004308C00D4
:100FD00039308E0021009513803022009D000430AE
:100FE0009E00270016131517141302302000C500A9
:100FF0000030C6008B31702387318B150800023416
:10169C0021008E150E16080021008E150E1608005E
:1016AC0081302200970008001630210097000800B6
:1016BC0020004608E2004508E1000800200046082A
:1016CC00E6004508E500080020004608E40045084F
:1016DC00E300080020004608EA004508E90008007D
:1016EC0020004608E8004508E70008007A30210091
:1016FC009900980122009601080004302000B000E7
:10170C008F313F278B31080005302000B0008D3120
:10171C004F258B310800D03021009E009B019C018D
:10172C0001309D000800183020009B009A01911098
:10173C0005309C0008002700161FA52BA62BA92BF3
:10174C008C3108248B31080001302000B000FA30B5
:10175C00B600863160268B3108003C3026009A009A
:10176C001830980099013F3025009E050800200094
:10177C00CC00111EC22BC32BBF2B4C0823009A008C
:10178C0008006400800101310130FE020030FF3B93
:10179C007F087E04031DC82B00342000C9010030D3
:1017AC008E31EC268B3120004E08C8008D31F82587
:1017BC008B3108002000C90101308E31EC268B31B1
:1017CC0020004E08C8008D31F8258B310800200010
:1017DC00C50045082300910015139513151400003E
:1017EC000000230013080800200093116708680408
:1017FC000319012C022C072C68088A0067080A00C0
:10180C008C310800200069086A0403190E2C0F2C77
:10181C00142C6A088A0069080A008C3127001613F8
:10182C0008002000C90100308E31EC268C312000DC
:10183C004F08C9004E08C8008D3136258C31080080
:10184C002000C90101308E31EC268C3120004F086C
:10185C00C9004E08C8008D3136258C310800200097
:10186C00C501111E3A2C3B2C432C23009E1E3F2CF1
:10187C00402C432C01302000C500200045080800F6
:10188C0021008E110032003221000E16003200327F
:10189C0020000E1E522C532C4E2C21008E15003283
:1018AC000032080021008E110032003221000E1689
:1018BC000032003220000E1E642C652C602C21009E
:1018CC008E1500320032080021008E150E162000F5
:1018DC000E1E712C722C6D2C0032003221008E11D8
:1018EC000032003221000E120032003208002100BA
:1018FC008E150E1620000E1E842C852C802C00328A
:10190C00003221008E110032003221000E12003202
:10191C000032080002302000B0002430CE0090309D
:10192C00CF008C3117248C3120002D08D8002C08C6
:10193C00D7008D31D9258C31080003302000B00040
:10194C001B30CE009030CF008C3117248C312D30D1
:10195C002000CE009030CF008C3126248C31080032
:10196C007C3028009D009C012000931121009315D0
:10197C0003302000C5000030C6008B3176238C313B
:10198C00273028009E0008008B3152238C31220016
:10199C000E128E1108308F3115278C310630200035
:1019AC00C9003030890BD82CC90BD82C000008008A
:1019BC002000CA004908CB004B08C5004A088E31EC
:1019CC007C268C3120004808CB004B08C5004A0807
:1019DC00013E8E317C268C31080000302000C50081
:1019EC00C6008D31A0258C3121009D01220097016C
:1019FC004030270095008C31CA248C3122008C1683
:101A0C00630008002000C7008C317D248D317C30B0
:101A1C00873161278D314030873161278D3120002E
:101A2C004708873161278D318C3158248D3108005E
:101A3C0001308E3159268D31200021084706031DB7
:101A4C00292D2008460603192C2D2D2D352D210866
:101A5C00C9002008C80001308C31DE248D3108000B
:101A6C00442D480884004908850000088D3108255C
:101A7C008D3101302000C8070030C93D20004808D6
:101A8C008400490885001200031D4D2D4E2D372D65
:101A9C00080000302000CE009030CF008C3117248D
:101AAC008D313C302000CC002108CE002008CD0028
:101ABC00853173258D313C302000CE008B31E023F5
:101ACC008D3108008731D0278D318B317C238D31BE
:101ADC008B315A238D318B3156238D318C31B62479
:101AEC008D318B3191238D318B31B3238D318B31F2
:101AFC0099238D318E31C6268D3108000630200099
:101B0C00B0001230CE009030CF008C3117248D31C4
:101B1C0051302000CE009030CF008C3126248D31F6
:101B2C0006302000BC00BD013C30C8008D31F825CA
:101B3C008D31080020004608C8004508C700C8368B
:101B4C00C70CC836C70C470826009800200045086B
:101B5C000339C7000430C735890BB12D26001A088C
:101B6C00CF392000470426009A0008002000D90035
:101B7C005E30CE009030CF008C3126248D313C303D
:101B8C002000CC005908D700D8015708CD005808C0
:101B9C00CE00853173258D3140302000C8008D3149
:101BAC00F8258D3108003C302000CC005808CE00C0
:101BBC005708CD00853173258D3120004208C300B4
:101BCC004108C2002E30C1003D30CE008B31E023E5
:101BDC008D3169302000C8009030C9008D31362518
:101BEC008D31080020004808C9000F2E48088600D7
:101BFC00870101088D3108258D3101302000C8077F
:101C0C0049084802803A783E031C0D2E0E2E0F2EEA
:101C1C00172E4808860087010108031D162E172E63
:101C2C00FC2D08002000C901CA01451C1E2E1F2EC8
:101C3C00232E4708C9074808CA3D0130C735C80DCF
:101C4C00890B242E0130C636C50C890B292E45086C
:101C5C004604031D322E332E1B2E4A08C60049089B
:101C6C00C50008002000C8004808C700C70DC70DF4
:101C7C0021001D08200047068339470621009D00DE
:101C8C001D140630890B482E003221009D149D181E
:101C9C00502E512E4D2E1C082000C60021001B0872
:101CAC002000C50008002000CC004C088B31ED232F
:101CBC008E312000C800C9014808CA004908CB0071
:101CCC000830CA35CB0D890B672E4C08013E8B3181
:101CDC00ED238E312000C800C9014808CA07490805
:101CEC00CB3D4B08C7004A08C60008002000C600C0
:101CFC00460823009100200045082300930095130B
:101D0C00151315150B0D0B0D01392000C7008B1386
:101D1C00553023009600AA30960095149518972EEE
:101D2C00982E942E15112000470C031C8B130318AE
:101D3C008B170800F9008C316A248E317C308F317E
:101D4C00CC278E3100308F31CC278E3179088F31F2
:101D5C00CC278E318C3146248E317908FC3903190D
:101D6C00B82EB92EBD2E2830890BBA2EC52E0B30AD
:101D7C00F8006230890BC02EF80BC02E0032080020
:101D8C00083023009F0090309D0024309E00A0302E
:101D9C009B0001309C0000302000C5000030C600C4
:101DAC008B3164238E3100302000C5000030C6001A
:101DBC008B316A238E3100302000C5000030C60004
:101DCC008B315E238E312000BB0108002000CB003C
:101DDC0002308F3115278E310B302000CA00623053
:101DEC00890BF62ECA0BF62E000020004B080319A7
:101DFC00002F012F092F4908C03ECC0000300318DA
:101E0C000130CD00102F4908803ECC000030031863
:101E1C000130CD004C088F3115278E310800200081
:101E2C00C8008C317D248F317C30873161278F3114
:101E3C000030873161278F312000480887316127B6
:101E4C008F318C3158248F3120004808FC3903190C
:101E5C00302F312F352F2830890B322F3E2F0B305E
:101E6C002000C7006230890B392FC70B392F0000B7
:101E7C00080009302000CE009030CF008C311724A0
:101E8C008F31023020006B06031D4D2F4E2F562F25
:101E9C003630CE009030CF008C3126248F316A2F13
:101EAC006B03031D5A2F5B2F632F4830CE009030ED
:101EBC00CF008C3126248F316A2F3F30CE009030EA
:101ECC00CF008C3126248F3108002000C901CA01B3
:101EDC000130CB0022008C160032003222008C1212
:101EEC0000320032113020004B0203187E2F7F2F5E
:101EFC008C2F0130C935CA0D890B802F0C0E01397E
:101F0C00C700C8014708C9074808CA3D0130CB07BC
:101F1C001A304B02031C932F942F702F4A08C600C3
:101F2C004908C500080020004508460403199F2FE6
:101F3C00A02FC72F0130C900AA2F0130C535C60DFF
:101F4C00890BA42F0130C907C61FAD2FAE2FA32FAD
:101F5C0046084802031DB42F45084702031CB72F3F
:101F6C00B82FBC2F4508C7024608C83B0130C636FF
:101F7C00C50C890BBD2F0130C902031DC62FC72FFD
:101F8C00AE2F4808C6004708C5000800F600803090
:101F9C00F700E82F21000E12770876050319D72FCA
:101FAC00D82FDA2F8E15DB2F8E1100320032031052
:101FBC00F70C21000E1620000E1EE52FE62FE12F48
:101FCC00003200327708031DEC2FED2FD02F2100AB
:101FDC000E128E150032003221000E1620000E1E3D
:101FEC00F82FF92FF42F0032003221000E1200329C
:101FFC0000320800533465346E347334203420348A
:10200C0020342034003456346F346C3475346D34D1
:10201C00653420342034003453346C3465346534E6
:10202C00703420343F34203400345534413452342D
:10203C0054342034543478342034003442346134F1
:10204C007434743465347234793420340034533439
:10205C0045344E344434203420342034303400346D
:10206C0020342034203420344C346F3475346434B0
:10207C00003420342034203420344D3475347434FE
:10208C0065340034203420344D3465346434693480
:10209C0075346D340034203420345034753473343A
:1020AC00683420340034533445344E3444340034D2
:1020BC00533454344F345034003443344E34543449
:0A20CC0000343A3400345634003476
:020000040001F9
:04000E00E43FFF3E8E
:00000001FF
